:020000040000FA
:100000005428112011201120213086000610B22022
:10001000283016200C30162004301620013016200F
:100020000800313086000610B2200800B300F03915
:10003000013886000610C420330EF03901388600DE
:100040000610C420BB200800C03016200800B300F2
:10005000F039033886000610C420330EF039033817
:1000600086000610C4200800C10105183428083095
:10007000C200C920CC200314051C0310C10CCC20E5
:100080000000C20B3B280800113084001A30B40075
:10009000342041088000840AB40B482808000E2050
:1000A0007B2024208C200800830185018601831693
:1000B0000530850086018312012000309D20242018
:1000C00009309D20AC206428342041085A3C031D8F
:1000D000642834204108443C031D6428342041082E
:1000E000413C031D6428342041082C3C031D642836
:1000F00044204F20632811082720120827203A3077
:10010000272013082720140827203A302720150815
:1001100027201608272008001B0827201C08272056
:100120002D3027201E0827201F0827202D302720AC
:10013000230827202408272008008900A620FF394B
:10014000031908002720890A9E2808000313831634
:1001500008148312080808001430B400B220B40B4D
:10016000AE2808006230B1006430B200B20BB6288D
:10017000B10BB42808001230B1002130B200B20B2C
:10018000BF28B10BBD2808002230B100B10BC62832
:1001900008001530C300CF284130C3000000C30B56
:0401A000CF2808005C
:02400E00F13F80
:1042000047005000530020004E004D004500410083
:10421000000041006D004700200076002E003400B1
:044220006100000039
:00000001FF
